:1000000000308A000428000084011F30830570300E
:1000100083168F001F129F121B0880399B00073028
:100020009C001F129F121B0880399B0083121F1017
:10003000941283160611861406120030831294005F
:10004000831694000108C03981000B30F700073097
:1000500083128101813084000008F0390738800064
:1000600064000008F739F719F0397704800090012F
:100070000030F800920000308316920007309C0098
:10008000050864000630F700F70B44281C088312AB
:100090000D13FE3083169D0005158F010F086300B8
:04400E003D3FFC3FF7
:00000001FF
